:1000000017C031C030C02FC02EC084C22CC02BC03E
:100010002AC029C028C027C026C056C172C101020B
:100020000408102002020202020200000000360052
:1000300011241FBECFE5D2E0DEBFCDBF10E0A0E6A9
:10004000B0E0E0EBF8E002C005900D92A236B107F7
:10005000D9F720E0A2E6B0E001C01D92AF39B207A7
:10006000E1F77AD323C4CCCFCF9381E990E002D2D9
:10007000C82F813021F0823011F0833019F4C09301
:1000800060002DC0811103C08FEF88BD10C0843087
:1000900089F480E488BDCCE360E87BEB80E090E00D
:1000A00005D2C150C9F78FEF88BD1092670010923A
:1000B000620015C0853098F0809162008C1730F492
:1000C00018BC60E87EE380E090E0F0D18C2F809552
:1000D000809367008091670088BDC0936200CF91D4
:1000E0000895809160008130E1F5809163009091E6
:1000F0006400A0916500B0916600892B8A2B8B2B40
:1001000091F020916300309164004091650050911E
:10011000660068E970EE8EE090E024D3283018F095
:1001200069EF620F01C060E080916300909164000C
:10013000A0916500B0916600883D9E40A105B10583
:1001400068F48091630090916400A0916500B09183
:100150006600892B8A2B8B2B09F06FEF81E990E0E9
:1001600087D180916000823029F46091610081E93B
:1001700090E07ED180916000833029F4609162002C
:1001800081E990E075C1089588E087BB18BAB19BFA
:1001900006C0B49902C0C398FCCFC39AFACF8AE0D4
:1001A00087BB18BA60E681E990E060D164E370E053
:1001B00081E990E060D161E770E081E990E060D191
:1001C00083EF8ABD81E083BF8FEF88BD08955DD145
:1001D00080916200882319F120EF39E442E050E079
:1001E00061E084E01AD260936300709364008093AE
:1001F0006500909366008091630090916400A091E7
:100200006500B0916600892B8A2B8B2B19F4C39A59
:1002100084E102C0C3988AE0809361000895C39886
:100220008EE180936100109263001092640010923E
:10023000650010926600089510927C0010927D0077
:1002400010927B001092690010926A001092680070
:100250008093900087B3856087BBC29AC09AB89894
:1002600088EA8DB980EF8EB9089590916800903139
:10027000E1F3E0916A00F0E0E559FF4F808380915F
:100280006A008F5F8F7080936A00809168008F5F33
:1002900080936800089580917B008823E1F3E091CA
:1002A0007C00F0E0E258FF4F808190917C009F5FDE
:1002B0009F7090937C0090917B00915090937B0075
:1002C000089580917B0008951F920F920FB60F92B0
:1002D00011248F9310928F0010928E00B898B29BC9
:1002E00002C0B09BFCCFB09902C088EF01C088EA81
:1002F0008DB980EF8EB98F910F900FBE0F901F9028
:1003000018951F920F920FB60F9211242F933F93BF
:100310004F935F936F937F938F939F93AF93BF930D
:10032000EF93FF9380918E0090918F008230910522
:1003300009F459C028F4009761F0019779F185C05C
:100340008430910509F458C030F1059709F45DC077
:100350007CC08FB1882331F08FB186959091900049
:1003600089133EC0789B67C0E0919200F0919300A2
:10037000309739F080917B00882319F080917B00C1
:100380000995E0919400F0919500309709F0099556
:1003900081E090E052C08FB1811122C0809168004D
:1003A0008823D1F0E0916900F0E0E559FF4F8081AA
:1003B0008FB9809169008F5F8F7080936900809101
:1003C000680081508093680082E090E090938F00F5
:1003D00080938E00B89A17C0B8981FB88EE78EB970
:1003E00088EA8DB910C083E090E090938F008093ED
:1003F0008E00B8981FB827C085E090E090938F00DA
:1004000080938E00B89880E71FC080917B00803178
:1004100090F4E0917D008FB1F0E0E258FF4F8083CF
:1004200080917D008F5F8F7080937D0080917B0035
:100430008F5F80937B0084E090E090938F008093A7
:100440008E001FB8B89A8EE78EB9FF91EF91BF91D9
:10045000AF919F918F917F916F915F914F913F915C
:100460002F910F900FBE0F901F901895862FE4CEFE
:10047000862FFBCE10CF7093930060939200089567
:1004800070939500609394000895809192009091EC
:100490009300892B51F0759B08C013DF882329F046
:1004A000E0919200F091930009940895CF92DF9229
:1004B000EF92FF92CF93DF936B017C0175D0EB013C
:1004C000C114D104E104F10479F0DFDF6DD06C1BBD
:1004D0007D0B683E7340A0F381E0C81AD108E108A3
:1004E000F108C851DC4FECCFDF91CF91FF90EF9036
:1004F000DF90CF90089580B7807F80BF80B78068FD
:1005000080BF8CB580648CBD8FEF8DBD80B7876058
:1005100080BF08951F920F920FB60F9211242F9350
:100520003F938F939F93AF93BF9380919700909148
:100530009800A0919900B0919A003091960026E021
:10054000230F2D3730F029E8230F0396A11DB11D8D
:1005500003C00296A11DB11D2093960080939700C1
:1005600090939800A0939900B0939A0080919B007B
:1005700090919C00A0919D00B0919E000196A11DBC
:10058000B11D80939B0090939C00A0939D00B0931D
:100590009E00BF91AF919F918F913F912F910F90AE
:1005A0000FBE0F901F9018953FB7F89480919B0055
:1005B00090919C00A0919D00B0919E0022B708B63A
:1005C00001FE05C02F3F19F00196A11DB11D3FBFCF
:1005D0006627782F892F9A2F620F711D811D911D1B
:1005E00043E0660F771F881F991F4A95D1F708953A
:1005F0008AB582608ABD8AB581608ABD83B7887FEB
:10060000836083BF789489B7826089BF74DF86B1C5
:100610008877866886B9379A08958F929F92AF92AD
:10062000BF92CF92DF92EF92FF920F931F93CF93DF
:10063000DF93C82FD0E0FE01E25EFF4FE490FE01A1
:10064000EC5DFF4FC491611102C0F12C01C0FE2C82
:10065000CA01B90120E43FE140E050E0A7D0B90170
:10066000CA0120E83EE340E050E07CD0D0E0CC0F6F
:10067000DD1FC65DDF4F80E090E0DC01FE0165918B
:100680007491FB0160816E216F111FC04C015D01EF
:100690006FEF861A960AA60AB60A82179307A4076E
:1006A000B50709F447C0D501C401E8CF4C015D018D
:1006B000FFEF8F1A9F0AAF0ABF0A82179307A4079A
:1006C000B50709F437C0D501C401FE0165917491E5
:1006D000FB0160816E216F11E9CF89019A01081B2E
:1006E000190B2A0B3B0B60E070E0CB01FE01A591DA
:1006F000B491EC91EE21EF110AC0601771078207E7
:100700009307C1F06F5F7F4F8F4F9F4FEFCF28E070
:1007100032E540E050E04AD049015A01C501B40138
:100720006058714C8F4F9F4F20E43FE140E050E014
:1007300019D003C020E030E0A901CA01B901DF915E
:10074000CF911F910F91FF90EF90DF90CF90BF90CE
:10075000AF909F908F90089581B781BF49DF14DDDE
:1007600036DDFECFA1E21A2EAA1BBB1BFD010DC078
:10077000AA1FBB1FEE1FFF1FA217B307E407F50751
:1007800020F0A21BB30BE40BF50B661F771F881F2D
:10079000991F1A9469F760957095809590959B01C3
:1007A000AC01BD01CF01089568940013E894A0E066
:1007B000B0E0ECEDF3E01DC0EFEFE7F959016A019D
:1007C0005E23550FEE08FE2C87019B01AC019E2392
:1007D000990F660B762FCB013BD0CDB7DEB7EAE0A1
:1007E00024C02F923F924F925F926F927F928F928E
:1007F0009F92AF92BF92CF92DF92EF92FF920F93B0
:100800001F93CF93DF93CDB7DEB7CA1BDB0B0FB6B9
:10081000F894DEBF0FBECDBF09942A883988488876
:100820005F846E847D848C849B84AA84B984C8840C
:10083000DF80EE80FD800C811B81AA81B981CE0F03
:10084000D11D0FB6F894DEBF0FBECDBFED010895E8
:10085000DF93CF939F92A0E49A2E0024D001E00171
:10086000F00116950795F794E794D794C794B79439
:10087000A79448F41068A20FB31FC41FD51FE61F2A
:10088000F71F081E191E220F331F441F551F661F16
:10089000771F881F991F9A9421F79D01AE01BF0110
:1008A000C00111249F90CF91DF910895F894FFCF5C
:0208B000011E27
:00000001FF
